:03000000023AAE13
:0C3AAE0078FFE4F6D8FD75816E023AF551
:100F980020000A3C2E2E2E3E004950436F6E6E658F
:100FA80063745245510A004950436F6E6E6563740D
:100FB800000A49504E6F41434B210A003E432C56CC
:100FC8002C43432CC0E4E0EFF2E5F020D1E8EDEA51
:100FD800EEEC49500A003E432C4D41432C2530325B
:100FE80062583A25303262583A25303262583A25EA
:100FF800303262583A25303262583A2530326258D7
:101008002C4D414320E0E4F0E5F10A003E432C5624
:1010180045522C20332E3220EEF2202573202573E2
:101028002CC2E5F0F1E8FF20495020ECEEE4F3EBA8
:10103800FF0A0041707220313420323031300031E3
:10104800313A31303A3131003E432C4C442C505225
:101058004F473A2020202020202020202020202018
:101068002020202020202020202020202020202078
:101078002020202020202020202020202020202068
:101088002020202020202020202020202020202058
:1010980020202020202020202CC4E0F2E020EFF0A7
:1010A800EEF8E8E2EAE828F4E0E9EB290A003E2A4B
:1010B8002C312CCEF1EDEEE2EDFBE520EFE0F0E097
:1010C800ECE5F2F0FB20F1E5F2E5E2EEE3EE20E8F4
:1010D800EDF2E5F0F4E5E9F1E00A003E412C41309B
:1010E800312C2562752E2562752E2562752E256296
:1010F800752C495020E0E4F0E5F120E0E4E0EFF25F
:10110800E5F0E00A003E412C4130322C2562752E74
:101118002562752E2562752E2562752C495020E0B2
:10112800E4F0E5F120EEF1ED2E20F1E5F0E2E5F056
:10113800E00A003E412C4130332C2562752E256291
:10114800752E2562752E2562752C495020E0E4F035
:10115800E5F120F0E5E72E20F1E5F0E2E5F0E00A20
:10116800003E412C4130342C2562752E2562752EA7
:101178002562752E2562752CCCE0F1EAE020F1E5B8
:10118800F2E80A003E412C4130352C2562752E25A7
:1011980062752E2562752E2562752CD8EBFEE70A3E
:1011A800003E2A2C312CC4EEEF2E20EFE0F0E0ECCC
:1011B800E5F2F0FB20F1E5F2E5E2EEE3EE20E8ED02
:1011C800F2E5F0F4E5E9F1E00A003E422C53303153
:1011D8002C2562752CC6E4E0F2FC20E7E0EFF0EE87
:1011E800F1E020F1EEE5E4E8EDE5EDE8FF20EEF2D0
:1011F80020F1E5F0E2E5F0E00A003E422C533032FF
:101208002C2562752CCEE1ECE5ED20F120F1E5F01E
:10121800E2E5F0EEEC20E1E5E720EAE2E8F2E0EDD5
:10122800F6E8E90A003E422C5330332C2562752C2F
:10123800CFE5F0E5E7E0EFF3F1EA20EFF0E820EFA3
:10124800EEF2E5F0E520F1E2FFE7E820F120F1E534
:10125800F0E2E5F0EEEC0A003E422C5330382C2543
:1012680062752CCCE5E4EBE5EDEDFBE92049502077
:10127800EAE0EDE0EB28E7E0E4E5F0E6EAE020E488
:10128800EE203520F1E5EA290A003E422C5330359C
:101298002C2562752CCAE0EDE0EB20F8E8F0EEEAC8
:1012A800EEE2E5F8E0F2E5EBFCEDEEE3EE20EEE150
:1012B800ECE5EDE00A003E532C5330362C25303255
:1012C80062582530326258253032625825303262F1
:1012D80058253032625825303262582C4D4143200F
:1012E800E0E4F0E5F120F8E8F0EEEAEEE2E5F8E017
:1012F800F2E5EBFCEDEEE3EE20EEE1ECE5EDE00AE5
:10130800003E454E440A000A44756D70582020205E
:10131800202030302030312030322030332030341B
:1013280020303520303620303720303820303920F2
:101338003041203042203043203044203045203096
:1013480046000A3A003A20000A000A44756D7044C3
:1013580020202020203030203031203032203033FF
:1013680020303420303520303620303720303820B7
:101378003039203041203042203043203044203062
:101388004520304600457272206B65790052642012
:10139800656570726F6D0A005264204D454D0A00F4
:1013A800526420436F64650A00577269746520436C
:1013B8006F64650A0044656275674950204F4E0A9C
:1013C8000044656275674950204F46460A004465E7
:1013D80062756755736572204F6E0A0044656275C1
:1013E8006755736572204F46460A00446562756703
:1013F8004D7367204F6E0A0044656275674D7367C9
:10140800204F46460A00436F6E666967206C6F631B
:101418006B210A00577220656570726F6D0A002093
:101428005361766520656570726F6D210A0045729B
:1014380072204D414321004C6F61643E3E002A00FA
:10144800CEF8E8E1EAE00A00202D20257528257568
:10145800290A003C4130313D003C4130323D003CDE
:101468004130333D003C4130343D003C4130353D56
:10147800003C21003C5330313D003C5330323D00AC
:101488003C5330333D003C5330353D003C533038FD
:081498003D003C5330363D00DD
:0645CD00010B00010900D2
:10459000C28E438910758BFF758DB7D2ABD28E2238
:03001B00023A1E88
:103A1E00C0E0C083C082C0D0C28E758BFF758DB7DB
:103A2E0020060675A61E75A6E10509D202E50B60F5
:103A3E0002050B050EE50E540F7051E50AD39401E5
:103A4E004002150AD20EE50E543F7012D200907A43
:103A5E00F9E0600A04F0E0D394B44002D206907A02
:103A6E00F2E0600204F090756FE0600214F0907A5C
:103A7E00FAE0D394014003E014F0300502050CE5A2
:103A8E000DD394644004D2068002050DE508D3944C
:103A9E000140021508D28ED0D0D082D083D0E03231
:10091100C291C290D2B5C20B7D027C007F07124505
:10092100598F25E525646060097D017F601244F4DB
:10093100D20BE4FDFC7F0B1245598F25E52530E6EE
:10094100097D04E4FF124518D20B7D017C007F076D
:100951001245598F25E5257008FD7FFF1244F4D219
:100961000B300B03126000C288C2A8C2AA758900AD
:10097100123EE69077AAE0B4FA06A3E064CE607B6B
:10098100E4F52574A22525F582E43477F583E4F0B6
:100991000525E525B443EC9077AA74FAF0A374CE4B
:1009A100F0A374CCF09077B0740AF0E4A3F0A30440
:1009B100F0A3F09077A674FFF0A3F0A3F0E4A3F006
:1009C1009077C17403F0E4F525E5252401FFE433B4
:1009D100FE74A22525F582E43477F583E0FD124407
:1009E100D00525E525C3944340DFE4F5A775A61E90
:1009F10075A6E1907FF0F0A3F080FE9077B57403C7
:100A0100F0A374CCF0E49077B4F0907AF7F0A3F00F
:100A110012347FC2B5123646C206124241D20BC20F
:100A21000DC20C9079E27408F09077207424F0E400
:100A3100A3F09077AAE0907722F09077ABE09077DF
:100A410023F09077ACE0907724F09077ADE0907749
:100A510025F09077AEE0907726F09077AFE0907731
:100A610027F0750A01E49079E3F0C207C208C209D0
:100A7100C20A1244A9200B19AF257E007D0312354D
:100A810065E4FF1238CD7E0F7F98E4FBFDFC123048
:100A9100A4907AF9E060037401F0E490756FF0F5C9
:100AA1000C9079E1F0F50D12459075A70775A61E1A
:100AB10075A6E1D2AFE4F50D90756FE07003121BDE
:100AC100FE907AFAE06401701D9080007410F0903D
:100AD10080A874FFF0A3F0A3F0A3F0E4907AFAF0F9
:100AE100D20BC20CC20D908008E0F52530E405D28E
:100AF100077410F0E52530E508D2099080087420CC
:100B0100F0E52530E608D2089080087440F0E50C45
:100B1100C394034019908002E4F0908001F090802A
:100B210000F0E50C94064006E4F50C124241908079
:100B3100A0E070031240579080B8E07003123F6448
:100B41009080D0E070031241E5908000E070133096
:100B510007101231AB90779DEFF0D3940040031250
:100B61000026908002E07006908000E06005D205CA
:100B7100020AB6C205E4F50C90756FE06003020A43
:100B8100B6200B129079E4E0600C7E0F7F9A12324E
:100B9100AFE49079E4F0300912122DD890779DEFEF
:100BA100F0D394004005E0FF1245A0200803020D98
:100BB1003A122C5190779DEFF07003020AB69077AC
:100BC100E1E054BF247F7003020C95147003020C02
:100BD1006D24026003020CDC200B077E0F7FA11243
:100BE10032AF200F03020D3A9077B9E0700690778B
:100BF100BDE06067907AEEE0FF9077B9E0B5072439
:100C0100907AEFE0FE9077BAE0B50618907AF0E0BE
:100C1100FE9077BBE0B5060C907AF1E0FE9077BCD0
:100C2100E06E60379077BDE06F6003020D3A907A15
:100C3100EFE0FF9077BEE06F6003020D3A907AF02B
:100C4100E0FF9077BFE06F6003020D3A907AF1E028
:100C5100FF9077C0E06F6003020D3AC2039079E321
:100C61007401F0120021750A01020D3A907AF9E03F
:100C710060037401F0907AE6E0FF9077E3E06F6043
:100C810003020D3A907AE6E004F0E4F50A9079E186
:100C9100F0020D3A300303020D3A9077B0E0700391
:100CA100020AB690771FE060089077C1741EF08049
:100CB100069077C17403F01245D4D203E4F50A908B
:100CC10079E1F0907AF204F0E4907AE5F0A3F02073
:100CD1000B677E0F7FAF1232AF805E907AF9E060D2
:100CE100037401F03003529077E1E020E74B9077F5
:100CF100E3E0FF907AE5E0FE6F600D907AEDE07041
:100D010007EE146F70338013907AE5E004F090776A
:100D11009DE0FFD39404400312437690746B748278
:100D2100F0A37401F09077E3E090746DF07E747F2E
:100D31006B7D03123C4D020AB6200303020E58E5F7
:100D41000A706E124420EF60237E787FE19078E292
:100D5100E02404FD123C4D907AEDE070099077C1DA
:100D6100E0F50A020AB6E4F50A020AB6907AF2E060
:100D7100D3943C403C907AEDE0703690771FE07060
:100D810030907AF204F01245BAE49078E1F0A3745D
:100D910012F0907AE6E09078E3F0A374FDF090759C
:100DA1007063A2019078E563A2017F1212299F80EE
:100DB100981245AF8F25E525B4011590746B7483A6
:100DC100F0E4A3F07E747F6B7D02123C4D020AB603
:100DD100E525D39401401C90746B7483F0A37401D6
:100DE100F0E52524FEA3F07E747F6B7D03123C4D5C
:100DF100020AB6E50A64016003020AB69079E1E0ED
:100E010004F0200B077E0F7FB91232AF9077C1E05B
:100E1100C3941E5004E02402F09079E1E0C39405EC
:100E2100400DC203E49079E3F0120021020AB67C7E
:100E31007A7DEE9077B5E0FAA3E0FB7F02123DDE0A
:100E41007E787FE19078E2E02404FD123C4D9077BA
:100E5100C1E0F50A020AB6E50A64016003020AB6B6
:100E61009079E3E014604624FE6042147003020F9F
:100E71004B24046003020AB6E4F50C200F139079A9
:100E8100E37404F09079E1E05401F0750A01020A7B
:100E9100B69080027410F0E49079E3F09079E10467
:100EA100F0750A12907AEE74FFF0020AB6907AEEAB
:100EB100E07003020F359078E17480F09078E3746C
:100EC10001F0E4A3F0A304F0A37430F0A3747BF069
:100ED100E4F52574E82525F582E43478F583747DFD
:100EE100F074E92525F582E43478F583E4F0E5250D
:100EF10024079078E2F07C7A7DEE9077B5E0FAA352
:100F0100E0FB7F02123DDE7E787FE1E5252409FDCD
:100F1100123C4D907AEDE0601B1245D4D203E4F50A
:100F21000A9079E1F0907AF204F0E4907AE5F0A386
:100F3100F0020AB6300F07E49079E3F08006907969
:100F4100E37404F0750A12020AB69080027410F07C
:100F5100750A039079E1E06401FFF09079E374018F
:100F6100F0EF70199077BDE06013FCA3E0FDA3E002
:100F7100FEA3E0FF907AEE1222F8020AB69077B94A
:100F8100E0FCA3E0FDA3E0FEA3E0FF907AEE1222D5
:060F9100F8020AB680FE22
:010F97002237
:100026009077E2E0B444047F0180027F009077E19C
:10003600E0B447047E0180027E00EE5F604A90775E
:10004600AAE09077E3F09077ABE09077E4F09077D2
:10005600ACE09077E5F09077ADE09077E6F09077BA
:10006600AEE09077E7F09077AFE09077E8F09077A2
:10007600E27452F090771963A2019080A863A201FE
:100086007F0612299F02090790779DE0C3940850C6
:10009600030209109077AAE0FF9077E3E06F600310
:1000A6000209109077ABE0FF9077E4E06F600302FF
:1000B60009109077ACE0FF9077E5E06F60030209E6
:1000C600109077ADE0FF9077E6E06F6003020910CD
:1000D6009077AEE0FF9077E7E06F6003020910903B
:1000E60077AFE0FF9077E8E06F6003020910907742
:1000F600E2E06444701A9080A8E0B4FF1390771988
:1001060063A2019080A863A2017F0612299F801036
:1001160090771DE09080ACF090771EE09080ADF077
:10012600907AF9E060037401F0907AFA7464F090C2
:1001360077E27452F09077E1E0646D60030202AA00
:100146007BFF7A0F79C41219047BFF7A0F79DE9050
:1001560077AAE0F52EA3E0F52FA3E0F530A3E0F5AE
:1001660031A3E0F532A3E0F533121904752EFF75BD
:100176002F1075303B7531FF7532107533477BFF95
:100186007A1079141219047BFF7A10795012190427
:100196007BFF7A1079B61219047BFF7A1079E39007
:1001A60077B0E0F52EA3E0F52FA3E0F530A3E0F558
:1001B600311219047BFF7A11790D9077B9E0F52E8B
:1001C600A3E0F52FA3E0F530A3E0F5311219047B87
:1001D600FF7A11793B9077BDE0F52EA3E0F52FA3CA
:1001E600E0F530A3E0F5311219047BFF7A11796945
:1001F6009077A6E0F52EA3E0F52FA3E0F530A3E077
:10020600F5311219047BFF7A11798C9077A2E0F50B
:100216002EA3E0F52FA3E0F530A3E0F53112190483
:100226007BFF7A1179A91219047BFF7A1179D2A280
:100236000FE433F52E1219047BFF7A127902907AB5
:10024600EDE0F52E1219047BFF7A12792D907AF9DA
:10025600E0F52E1219047BFF7A12796090771FE081
:10026600F52E1219047BFF7A127992A201E433F576
:100276002E1219047BFF7A1279BE907AE7E0F52EEA
:10028600A3E0F52FA3E0F530A3E0F531A3E0F532C6
:10029600A3E0F533121904123B3A7BFF7A1379096E
:1002A600121904229077E1E0644C70737E137F0F7D
:1002B600FBFDFC1230A49077E9E0F526A3E0F527D4
:1002C600E4F529E5269077EBF0A3E527F07E137F8A
:1002D6004A7C777DEB7B021230A4E4F528852782E1
:1002E600852683E0FF74EB2528F582E43477F583D1
:1002F600EFF00527E527700205260528E528B41046
:10030600DC7E137F4D7C777DEB7B101230A40529B4
:10031600E529C3941040AC7E137F501232AF229071
:1003260077E1E0646C7060F52A7E137F52FBFDFC7A
:100336001230A4E4F529E49077EBF0A3E52AF07EE9
:10034600137F4A7C777DEB7B021230A4E4F528A864
:100356002AE6FF74EB2528F582E43477F583EFF07F
:10036600052A0528E528B410E67E137F4D7C777DA7
:10037600EB7B101230A40529E529C3940840B77E0B
:10038600137F501232AF229077E1E0644B7061F533
:100396002874D32528F582E43477F583E060327437
:1003A600D32528F582E43477F583E0F4602374D30B
:1003B6002528F582E43477F583E0FF74E92528F5EE
:1003C60082E43477F583E0B507100528E528B408FC
:1003D600C090756F7432F00209079077E17421F0CE
:1003E600300B030209077E137F8D1232AF02090715
:1003F6009077E1E0B4521A200B077E137F951232F4
:10040600AF9077E17472F07E777FE17D08123BC68C
:10041600229077E1E064497045200B077E137FA0A8
:100426001232AF9077E9E0F526A3E0F527E4F52848
:10043600852782852683E0FF74EB2528F582E43440
:1004460077F583EFF00527E527700205260528E5F1
:1004560028B480DC7E777FE17D8A123BC6229077C6
:10046600E1E064437046200B077E137FA81232AF8B
:100476009077E9E0F526A3E0F527E4F528852782BD
:10048600852683E493FF74EB2528F582E43477F51B
:1004960083EFF00527E527700205260528E528B431
:1004A60080DB7E777FE17D8A123BC6229077E1E092
:1004B600645A7053200B077E137FB11232AF9077C8
:1004C600E9E0F526A3E0F5277C777DEB7B80AF2777
:1004D600AE261243ECE4F528852782852683E4932D
:1004E600FF74EB2528F582E43477F583EFF00527D2
:1004F600E527700205260528E528B480DB7E777F90
:10050600E17D8A123BC6229077E1E06444600302F3
:10051600059E9077E9E0FF64447003020907EFB493
:10052600310CC20B7E137FBD1232AF0209079077E2
:10053600E9E0B4300CD20B7E137FC91232AF020948
:10054600079077E9E0B4320CD20C7E137FD61232D4
:10055600AF0209079077E9E0B4330CC20C7E137F33
:10056600E41232AF0209079077E9E0B4340CD20DF9
:100576007E137FF31232AF0209079077E9E0B435B4
:100586000CC20D7E147F001232AF0209079077E984
:10059600E0FF12001E02090790756FE07013200B32
:1005A600077E147F0E1232AF9077E17421F00209B4
:1005B6000790756F7432F09077E1E0FFB45104C292
:1005C600AF80FEEF64577045200B077E147F1C1228
:1005D60032AF9077EAE090779DF0E4F52890779D2A
:1005E600E0FFE528C39F400302090774EB2528F5C1
:1005F60082E43477F583E0FF9077E9E02528241834
:10060600F582E43476F583EFF0052880D09077E123
:10061600E0645360030206C1200B077E147F271295
:1006260032AF9077AAE0FF907621E06F703C90772A
:10063600ABE0FF907622E06F70309077ACE0FF90F1
:100646007623E0B507249077ADE0FF907624E0B5F9
:1006560007189077AEE0FF907625E0B5070C907707
:10066600AFE0FF907626E06F60169077E17421F098
:10067600300B030209077E147F361232AF020907D8
:10068600E4F528E4F50DAF28FE74182528F582E474
:100696003476F583E0FD1244D00528E528C394FEA0
:1006A60040E1C2AFE4907FF0F0A3F0907FFD74AA22
:1006B600F0A374FFF0A37455F080FE9077E1E06438
:1006C6004F705A9077E9E0F526A3E0F527E5274530
:1006D60026700A200B077E147F3F1232AF200B07CD
:1006E6007E147F461232AFE4F52874EB2528F58296
:1006F600E43477F583E0852782852683F00527E5B0
:1007060027700205260528E528B480DE907AF8E0F1
:100716002480F0907AF7E03400F00209079077E140
:10072600E0644570749077E9E0FEA3E0FF907FF007
:10073600EEF0A3EFF0D39400EE94044038907FF0EF
:10074600E0FEA3E0FF907AF7E0FCA3E0FD9FEC9EBD
:100756004023E42FFFEE3401FED3ED9FEC9E5015AF
:10076600C2AF907FFD74AAF0A374FFF0A37455F096
:10077600E4F5A780FE7E147F481232AF7BFF7A1421
:100786007950907FF0E0F52EA3E0F52F907AF7E010
:10079600F530A3E0F5311219049077E1E064656065
:1007A600030209109077E9E0FFA3E0907FF0CFF015
:1007B600A3EFF0E4F526F527D3907FF1E095279097
:1007C6007FF0E095264020E4F50D2527FFE5263449
:1007D60001FE852782852683E0FD1244D00527E5A4
:1007E600277002052680D17E147F5B123CD4EF4E23
:1007F60060201200039077B0EFF01200039077B1FB
:10080600EFF01200039077B2EFF01200039077B387
:10081600EFF07E147F61123CD4EF4E60201200038D
:100826009077B9EFF01200039077BAEFF012000359
:100836009077BBEFF01200039077BCEFF07E147F49
:1008460067123CD4EF4E60201200039077BDEFF0A4
:100856001200039077BEEFF01200039077BFEFF01F
:100866001200039077C0EFF07E147F6D123CD4EF38
:100876004E60201200039077A6EFF01200039077E7
:10088600A7EFF01200039077A8EFF012000390771D
:10089600A9EFF07E147F73123CD4EF4E6020120055
:1008A600039077A2EFF01200039077A3EFF0120007
:1008B600039077A4EFF01200039077A5EFF0E4F52C
:1008C60028E4F50DE5282401FFE433FE74A225286B
:1008D600F582E43477F583E0FD1244D00528E52857
:1008E600C3944340DCC2AFE4907FF0F0A3F0907F66
:1008F600FD74AAF0A374FFF0A37455F0E4F5A78085
:0A090600FE7E777FE17D08123BC6FC
:0109100022C4
:1043B400AE07EEC39430400BEED394395005EE248F
:1043C400D0FF22EEC39461400BEED394665005EE09
:1043D40024A9FF22EEC39441400BEED3944650052A
:0843E400EE24C9FF22AF0622FE
:10457600907718E004F07006907717E004F09077D3
:0A45860017E0FEA3E0FF12453C22FF
:100003001245761243B4EFC454F0FEC0061245768F
:080013001243B4D0E02FFF22DC
:10418800E4907C53F0124576907C54EFF0C3943061
:104198004018E0FFD394395011907C53E02470F517
:1041A80082E43475F583EFF08011907C53E024703D
:1041B800F582E43475F583E4F0800C907C53E004D8
:1041C800F0E0D3940840BE752D00752E00752F00C1
:0C41D800E4F5307B017A757970122AAD95
:0141E40022B8
:043CD4008E2B8F2C78
:103CD800907717E4F0A374FFF0124576EF606EF466
:103CE800606B852C82852B83E493B507EC752D01D9
:103CF800E52C252DF582E4352BF583E4936025909A
:103D08007718E0252DFF907717E03400FE12453C28
:103D1800E52C252DF582E4352BF583E493B50704CE
:103D2800052D80CCE52C252DF582E4352BF583E493
:103D38009370A6E52D24FFFFE434FFFE907718E08A
:103D48002FF0907717E03EF07E007F0122E4FEFF1F
:013D58002248
:10347F007E147F79123CD4EF4E70037F01227E14AD
:10348F007F7C123CD4EF4E600C124576EF24D02493
:10349F00FF920F8002D20F7E147F82123CD4EF4E28
:1034AF00600C124576EF24D0907AEDF08005E49011
:1034BF007AEDF07E147F88123CD4EF4E600C1245EB
:1034CF0076EF24D0907AF9F08005E4907AF9F07EC7
:1034DF00147F8E123CD4EF4E600C124576EF24D041
:1034EF0024FF92018002C2017E147F94123CD4EF1C
:1034FF004E600C124576EF24D090771FF08005E4D4
:10350F0090771FF09077AA63A201907AE763A201E8
:10351F007F0612299F30013B7E147F9A123CD4EF15
:10352F004E6030120003907AE7EFF0120003907AAA
:10353F00E8EFF0120003907AE9EFF0120003907AAF
:10354F00EAEFF0120003907AEBEFF0120003907A9B
:06355F00ECEFF07F0022FA
:1042E6009079E2E0C3947C40027F0A9079E2E0FE96
:1042F60004F074202EF582E43477F583EFF0BF0ADC
:10430600279079E2E0FF04F074202FF582E43477F9
:10431600F583E4F09079E2E0FF123D599079E2747A
:0943260008F0907721E004F02278
:104241009080007480F09077A263A201F583F582DB
:1042510063A2017F0812299F9077AA63A20190802F
:104261008863A2017F0A12299F9080927407F0A3AC
:1042710074D0F0A37406F09077B4E0FF9080B1F0B1
:104281009080E1EFF09080957455F0A3F09080005C
:0A4291007401F090800974F0F0222F
:10405700908009E04410F09080A0E070609080A10B
:104067007482F09080A874FFF0A3F0A3F0A3F07F10
:10407700039080AEEFF0A374CBF09080007402F051
:10408700907C4712230400000000907C47E090805A
:1040970040F0907C48E0908041F0907C49E090802F
:1040A70042F0907C4AE0908043F0A3E4F0A3F0A3B1
:0D40B700F0A3F0908018F0A3F0A3F0A3F0A8
:0140C40022D9
:1041E500908009E04440F09080D17482F07F039084
:1041F50080DEEFF0A374CCF09080027402F0907C26
:104205004B12230400000000907C4BE0908058F096
:10421500907C4CE0908059F0907C4DE090805AF075
:10422500907C4EE090805BF0A3E4F0A3F0A3F0A3B4
:0B423500F0908030F0A3F0A3F0A3F0A5
:01424000225B
:103F6400908009E04420F09080B8E0706C9080B9B3
:103F74007482F07F039080C6EFF07FCDA3EFF07FD3
:103F8400039080C4EFF0A374CDF09080C074FFF070
:103F9400A3F0A3F0A3F09080017402F0907C4F1280
:103FA400230400000000907C4FE090804CF0907C53
:103FB40050E090804DF0907C51E090804EF0907CE9
:103FC40052E090804FF0A3E4F0A3F0A3F0A3F090AC
:093FD4008024F0A3F0A3F0A3F097
:013FDD0022C1
:103DDE008C268D27A907EAFDE975F018A424ACFFFF
:103DEE00E5F034808F82F583EDF0EBFDE975F01888
:103DFE00A4FFAEF024ACFBEE34808B82F583A3EDF2
:103E0E00F08527828C83E0FDEF24A8FFEE3480FE40
:103E1E008F82F583EDF08527828C83A3E08F828ECF
:103E2E0083A3F0852782852683A3A3E0FDE975F0A1
:103E3E0018A424A8FFE5F03480FE8F82F583A3A397
:103E4E00EDF08527828C83A3A3A3E08F828E83A3BC
:043E5E00A3A3F02208
:063BC6008D2BAB07AA06DF
:103BCC00908000E030E5079079E47401F022907C5D
:103BDC0047E0FCA3E0FDA3E0FEA3E0F52F8E2E8DC5
:103BEC002D8C2CAE02AF038E838F8263A201E52E47
:103BFC00540744C0F583852F8263A201AF2B122A90
:103C0C0011E4FCFDFEE52F252BF52FEE352EF52EC0
:103C1C00ED352DF52DEC352CF52C908040E52CF068
:103C2C00A3E52DF0A3E52EF0A3E52FF09080007412
:103C3C0020F0AF2FAE2EAD2DAC2C907C471222F87D
:013C4C002255
:063C4D008D26AB07AA065C
:103C5300908002E030E5079079E47403F022907CD1
:103C63004BE0FCA3E0FDA3E0FEA3E0F52A8E298D43
:103C7300288C27AE02AF038E838F8263A201E529CE
:103C8300540744D0F583852A8263A201AF26122A02
:103C930011E4FCFDFEE52A2526F52AEE3529F52952
:103CA300ED3528F528EC3527F527908058E527F0E2
:103CB300A3E528F0A3E529F0A3E52AF09080027498
:103CC30020F0AF2AAE29AD28AC27907C4B1222F806
:013CD30022CE
:0238CD008F2743
:1038CF00908001E030E5099079E47402F07F0022E6
:1038DF00907C4FE0FCA3E0FDA3E0FEA3E0F52B8E70
:1038EF002A8D298C28907AE763A201E52A54074490
:1038FF00C8F583852B8263A2017F06122A27E52B49
:10390F002406F52BE4352AF52AE43529F529E43583
:10391F0028F5289079E563A201E52A540744C8F5F4
:10392F0083852B8263A201AF27122A27E4FCFDFEB9
:10393F00E52B2527F52BEE352AF52AED3529F52927
:10394F00EC3528F52890804CE528F0A3E529F0A365
:10395F00E52AF0A3E52BF09080017420F0AF2BAE99
:0D396F002AAD29AC28907C4F1222F8AF271A
:01397C002228
:1031AB009081E0E0F5260526052605260526052651
:1031BB0005260526052605260526908010E0F5290F
:1031CB00A3E0F52AA3E0F52BA3E0F52C9081E1E039
:1031DB00F52605260526052605260526052605269C
:1031EB00052605260526908014E0F52DA3E0F52E87
:1031FB00A3E0F52FA3E0F530E52FB52B08E530B5AF
:10320B002C037F0022E4F526E52F540744E0F583D9
:10321B0085308263A2019077E163A2017F08122AB5
:10322B00579077E363A20190771963A2017F06128F
:10323B00299F9077E1E0F527A3E0F528E4F52690A8
:10324B0077E1E0702AA3E024F8F526E52F54074434
:10325B00E0F58385308274082582F582E43583F5A9
:10326B008363A2019077E163A201AF26122A57AEC6
:10327B0027E4FCFDE5302528F530E52F3EF52FED55
:10328B00352EF52EEC352DF52D908014E52DF0A374
:10329B00E52EF0A3E52FF0A3E530F090800074400D
:0332AB00F0AF265B
:0132AE0022FD
:102C51009081E6E0F52605260526052605260526AA
:102C610005260526052605260526908028E0F52956
:102C7100A3E0F52AA3E0F52BA3E0F52C9081E7E092
:102C8100F5260526052605260526052605260526FB
:102C910005260526052690802CE0F52DA3E0F52ECE
:102CA100A3E0F52FA3E0F530E4F526E52FB52B0AD7
:102CB100E530B52C05C208022DBDE52F540744F0BF
:102CC100F58385308263A2019077E163A2017F08D9
:102CD100122A579077E1E0F527A3E0F528E528458A
:102CE1002770099080027410F07F0022907AEEE044
:102CF100FFF460309077E3E06F6003022D84907AF7
:102D0100EFE0FF9077E4E06F7079907AF0E0FF9068
:102D110077E5E06F706D907AF1E0FF9077E6E06F14
:102D21006031805F9077E3E0907AEEF09077E4E0B5
:102D3100907AEFF09077E5E0907AF0F09077E6E026
:102D4100907AF1F09077E7E0FFA3E09077B5CFF0CC
:102D5100A3EFF09077E1E0702AA3E024F8F526E5EF
:102D61002F540744F0F58385308274082582F5825B
:102D7100E43583F58363A2019077E163A201AF2675
:102D8100122A57AE27E4FCFDE5302528F530E52F62
:102D91003EF52FED352EF52EEC352DF52DAF2CAE64
:102DA1002BAD2AAC29AB30AA2FA92EA82DD31222E4
:102DB100E740099080027410F07F002290802CE59A
:102DC1002DF0A3E52EF0A3E52FF0A3E530F09080E0
:062DD100027440F0AF2681
:012DD70022D9
:102DD8009081E3E0F5260526052605260526052625
:102DE8000526052605260526052690801CE0F529DA
:102DF800A3E0F52AA3E0F52BA3E0F52C9081E4E00D
:102E0800F526052605260526052605260526052672
:102E1800052605260526908020E0F52DA3E0F52E51
:102E2800A3E0F52FA3E0F530E4F526E52FB52B0A4E
:102E3800E530B52C05C209022F2EE52F540744E8CA
:102E4800F58385308263A20190746F63A2017F0EBF
:102E5800122A6D90746FE0F527A3E0F52890747737
:102E6800E0FFF4604A907AE7E0FEEF6E7079A3E045
:102E7800FF907478E06F706F907AE9E0FF90747952
:102E8800E06F7063907AEAE0FF90747AE06F7057B1
:102E9800907AEBE0FF90747BE06F704B907AECE0F7
:102EA800FF90747CE06F703FE490747EF08008902F
:102EB800747E74FFF0D2D990746FE0702AA3E02476
:102EC800F2F526E52F540744E8F583853082740E21
:102ED8002582F582E43583F58363A20190746F63DC
:102EE800A201AF26122A6DAE27E4FCFDE5302528A5
:102EF800F530E52F3EF52FED352EF52EEC352DF579
:102F08002DAF2CAE2BAD2AAC29AB30AA2FA92EA8F9
:102F18002DD31222E75006E5284527700990800135
:102F28007410F07F0022908020E52DF0A3E52EF0AC
:102F3800A3E52FF0A3E530F09080017440F0AF26B0
:012F48002266
:0432AF008E2D8F2EA3
:1032B300908000E030E5079079E47401F022907C7F
:1032C30047E0FCA3E0FDA3E0FEA3E0F5348E338DDD
:1032D300328C31E534FFE5335407FEE42FF530EE4D
:1032E30034C0F52F853082F5837423F00530E53043
:1032F3007002052F532FC7F582852F83740AF005BB
:1033030030E5307002052F532FC79077AA63A201CF
:10331300852F8385308263A2017F06122A117406EA
:103323002530F530E4352FF52F852D83852E8263E7
:10333300A201852F8385308263A2011229F5E4FC63
:10334300FDFE907C47E0F8A3E0F9A3E0FAA3E02FA9
:10335300FFEE3AFEED39FDEC38FCEF2408FFE43EC6
:10336300FEE43DFDE43CFC907C471222F8907C4750
:10337300E0908040F0907C48E0908041F0907C4960
:10338300E0908042F0907C4AE0908043F09080008F
:033393007420F0B3
:013396002214
:0A30A4008E2B8F2C8C2D8D2E8B2F80
:1030AE00908000E030E5079079E47401F022907C86
:1030BE0047E0FCA3E0FDA3E0FEA3E0F5358E348DE2
:1030CE00338C32E535FFE5345407FEE42FF531EE4F
:1030DE0034C0F530853182F5837423F00531E53146
:1030EE00700205305330C7F582853083740AF005BF
:1030FE0031E531700205305330C79077AA63A201D3
:10310E0085308385318263A2017F06122A117406EF
:10311E002531F531E43530F530852B83852C8263EE
:10312E00A20185308385318263A2011229F58F3683
:10313E00EF2531F531E43530F530E52F6017852D6B
:10314E0083852E8263A20185308385318263A2013D
:10315E00AF2F122A11E5362408252FF52FFFE4FC98
:10316E00FDFEE5352FF535EE3534F534ED3533F519
:10317E0033EC3532F532908040E532F0A3E533F092
:10318E00A3E534F0A3E535F09080007420F0AF3560
:0C319E00AE34AD33AC32907C471222F806
:0131AA002202
:023D59008F3F9A
:103D5B00908000E030E5079079E47401F022907CCC
:103D6B0047E0FCA3E0FDA3E0FEA3E0F5438E428D0C
:103D7B00418C40E543FFE5425407FEE42FFFEE3450
:103D8B00C090772063A201F5838F8263A201AF3FBE
:103D9B00122A11E4FCFDFEE543253FF543EE3542C7
:103DAB00F542ED3541F541EC3540F540908040E56D
:103DBB0040F0A3E541F0A3E542F0A3E543F090808A
:103DCB00007420F0AF43AE42AD41AC40907C471243
:023DDB0022F8CC
:013DDD0022C3
:063565008E2A8F2BAB053E
:10356B00908000E030E5079079E47401F022907CC4
:10357B0047E0FCA3E0FDA3E0FEA3E0F5318E308D28
:10358B002F8C2EE531FFE5305407FEE42FF52DEEA1
:10359B0034C0F52C852D82F5837423F0052DE52D94
:1035AB007002052C532CC7F582852C83EBF0052D6F
:1035BB00E52D7002052C9077AA63A201852C8385DB
:1035CB002D8263A2017F06122A117406252DF52D7B
:1035DB00E4352CF52C532CC7E52A852D82852C83BD
:1035EB00F0052DE52D7002052C532CC7F582852C8B
:1035FB0083E52BF0052DE52D7002052C532CC7E52B
:10360B0031240AF531E43530F530E4352FF52FE46C
:10361B00352EF52E908040E52EF0A3E52FF0A3E597
:10362B0030F0A3E531F09080007420F0AF31AE3074
:0A363B00AD2FAC2E907C471222F850
:013645002262
:10453C00A2AF9210C2AF438E2075D2028F828E83AF
:0C454C00E0FFE4F5D2538EDFA21092AF26
:014558002240
:1044D000E5D220E0FBA2AF9210C2AF43D2028F829E
:1044E0008E83EDF075D25063D250A21092AFE5D218
:0344F00020E0FBCE
:0144F30022A6
:103EE600E4FDED2401FFE433FE12453C74A22DF5FA
:103EF60082E43477F583EFF00DBD3FE6E4FDED2473
:103F06007FFFE433FE12453C74982DF582E4347548
:103F1600F583EFF074982DF582E43475F583E0703F
:103F26001B74982DF582E43475F5837420F074992A
:103F36002DF582E43475F583E4F080040DBD80BE72
:103F4600E4907617F0FDEDFF7E0012453C74182DC7
:0D3F5600F582E43476F583EFF00DBDFEE951
:013F6300223B
:0243EC008B2B19
:1043EE00A2AF9210C2AF85A22C53A2FE8E838F82F3
:1043FE0005A28C838D827409122A9BE52B53A2FE93
:10440E0043A220122A9D53A2DF852CA2A21092AFA6
:01441E00FF9E
:01441F00227A
:10455900A2AF9210C2AF8C838D82EF122A9B43A225
:0C45690020122A9D53A2DFA21092AFFF87
:014575002223
:0244F4008F2611
:1044F600A2AF9210C2AFE4F5838D827406122A9B96
:10450600E52643A220122A9D53A2DFA21092AF7F76
:0145160001A3
:014517002281
:024518008F26EC
:10451A00A2AF9210C2AFE4F5838D82740A122A9B6D
:10452A00E52643A220122A9D53A2DFA21092AF7F52
:01453A00017F
:01453B00225D
:1028C400A907E7FFA805EF93C3966008403B74FC93
:1028D4002FFF80F00F08EF93C3966008402B74FB22
:1028E4002FFF80E00F08EF93C3966008401B74FA33
:1028F4002FFF80D00F08EF93D3966008400B74F934
:102904002FFF80C01F1F1F1F1FEF54FEF80303F784
:10291400E893FC08E893FD08E893FE08E893FF2297
:1029240009E993C39D6008402974FB29F980F109E2
:10293400E993C39E6008401A74FA29F980E209E910
:1029440093D39F6008400B74F929F980D31919199E
:102954001919E9C313C313FF22740093F8ECC39845
:102964004024701F740193F8EDC3984019701474D7
:0E2974000293F8EEC398400E7009740393F8B6
:10298200EFC39840037F00227F0122EDF8E6F008B2
:10299200A3DFFA22EDF8E0F608A3DFFA22E0A36350
:1029A200A201F0A363A201DFF475A2002263A201D7
:1029B200F0A363A20122E0A363A201F0A363A20138
:1029C200E0A363A201F0A363A201E463A201F0A366
:1029D20063A201DFE175A20022E0A363A2016DFE02
:1029E200936CFDEE058393FC158363A201DFEA7508
:1029F200A200227F00E493A363A201F00F600CA364
:102A0200E583C2E3F58363A20180EA75A20022E0B6
:102A1200A363A201F0A3E583C2E3F58363A201DF0E
:102A2200EE75A20022E0A363A201F0A3E583C2E453
:102A3200D2E3F58363A201DFEC75A20022E0A36377
:102A4200A201F0A3E58344F8C2E5F58363A201DFA6
:102A5200EC75A20022E583C2E3F583E0A363A20141
:102A6200F0A363A201DFEE75A20022E583C2E4D2E5
:0A2A7200E3F583E0A363A201F0A3E3
:102A7C0063A201DFEC75A20022E58344F8F583E044
:102A8C00A363A201F0A363A201DFEE75A20022F9F9
:102A9C0022C002C004C00612FFF0D006D004D0023F
:012AAC002207
:10397D004572724C656E210A000A496E49503A0033
:10398D00205544502054696D654750530A00200A54
:10399D00495054696D653A2000200A44415441470D
:1039AD0052414D3A20002049676E6F72650A200022
:1039BD002043414E2054696D654750530A002054F1
:1039CD007261737353656E644552520A000ACEF8E4
:1039DD00C4EBE8EDFB43414E210A000A45727241EA
:1039ED00647243414E3A00205265496E697420431A
:1039FD00414E0A002043414E283029203E20544F8D
:103A0D00210A0020545520300A0020545520310A37
:013A1D0000A8
:03001E00E4FF22DA
:10448100C2A9438902758C48758A4875D90475DBC0
:104491004875DC4875DD4875DE48E4F5E9F5F9D283
:0844A100D9C2DAD28CD2DE226E
:10445300C2D9907B0FE07013E5E92419F5EB30D74F
:1044630006E5F904F5FB2285F9FB22E5E924C8F505
:0E447300EB30D706E5F904F5FB2285F9FB22B4
:10432F00C2D9907B0FE0702C302416E5E92432F5CA
:10433F00EB30D707E5F904F5FB800385F9FBC224C1
:10434F0022E5E92405F5EB30D706E5F904F5FB2264
:10435F0085F9FB22E5E92432F5EB30D706E5F904C0
:07436F00F5FB2285F9FB229A
:1044A900124481907B0FE0C394645006123E62125D
:1044B9004453120022D223E4F555907C27F0F544A9
:0744C900F559C224F557224A
:10437600EF24FCF544D3940D4010200B077E397FC3
:104386007D1232AFE4F544D221229077E563A20193
:10439600907C1763A201AF4412299FC221200B0D06
:0E43A6007E397F867C777DE5AB441230A42201
:0F45A000D3EF6480948D5006E55970028F592235
:101BFE0020D903021D02202303021D02E55960674E
:101C0E0090746F540FFF7D46122996E5466401705D
:101C1E003A90747EE0B4FF0ED225200B127E397FEF
:101C2E008D1232AF8009302506E4F559021D0212DD
:101C3E0044531240C5200B0D7E397F9B7C747D6F03
:101C4E00AB591230A4E4F559021D0212445312404E
:101C5E00C5200B0D7E397FA67C747D6FAB5912307B
:101C6E00A4E4F559021D02E5446055907C1BE02466
:101C7E0005F526D3940D4007E4F544D221807590E6
:101C8E007C17E526540FFF7D46122996E54630E770
:101C9E0002D224E5466401701A302517E549B401D5
:101CAE0012200B127E397FB37C747D6FAB591230CC
:101CBE00A480031240C5124453E4F544D22180346B
:101CCE00E556601E907AFB540FFF7D46122996E56D
:101CDE0046B401032025031240C5124453E4F556C1
:101CEE00801220190C907B0FE0C3946450031237BE
:101CFE0023124453122F498F26EF7003021E2BE43A
:101D0E00F557E54630E70AE549B41905D2D9021E62
:101D1E002B12432FE546B4010CD225200B077E393A
:101D2E007FBD1232AFE558C394C8501B30031874F0
:101D3E00102558F582E4347BF583E5262558F558B1
:101D4E007D46AF2612298D300121E54620E71C90F5
:101D5E0079E57D46AF2612298DAF261238CDEF706C
:101D6E000A200B077E397FCB1232AFE546548160D5
:101D7E0003021E2BE526D3940D4010300B03021EDA
:101D8E002B7E397FDA1232AF021E2BE548D3940731
:101D9E00401F300B03021E2B9075707D46AF26122E
:101DAE00298D7E397FE87C757D70AB261230A4803C
:101DBE006CE50F30E662907C42E0FF90415693FE58
:101DCE00547F65467052EFA3936548704B907C42EA
:101DDE00E0C313FF2429F582E4347CF583E07038E8
:101DEE00530F3F907C42E0FD7470250FF582E43472
:101DFE0061F583EEF0ED90415793FE7471250FF56A
:101E0E0082E43461F583EEF074292FF582E4347C9C
:101E1E00F5837401F0430F40AF26121F57300E1A90
:101E2E00300015907B0FE0C39464500C0557E557B6
:101E3E0094F04004C2AF80FEC20E200203021F5176
:101E4E00906001E004F07006906000E004F0E5554B
:101E5E006031D39401400415558028907C27E0040E
:101E6E00F0E0D39403400D200B077E397FF412323D
:101E7E00AF1244A9200B077E3A7F011232AFE4F570
:101E8E0055D223E5566003021F4F30223F907AFB56
:101E9E0004F0A37408F0A37480F0A37401F0A3748B
:101EAE0006F0907C12E0907B00F0907C13E0907B2B
:101EBE0001F0907C14E0907B02F0907C15E0907B1A
:101ECE0003F0E4A3F0A3F075560BC22230207290FB
:101EDE007C10E07035E5567031907AFB7442F0A3B9
:101EEE007408F0907C11E0907AFDF0907C16E090F2
:101EFE007AFEF0A37401F0755606200B077E3A7F2A
:101F0E00101232AF907C10E004F0907C10E064026E
:101F1E00702FE556702B907AFB7402F0A37408F0C4
:101F2E00907C11E0907AFDF0A3F0A37401F0755649
:101F3E0006200B077E3A7F171232AF907C10E0041A
:081F4E00F0C202122488C20057
:011F56002268
:10442000E558602CE49078E1F0A3E558F0907AE646
:10443000E09078E3F0A37419F0907B1063A20190F0
:1044400078E563A201AF5812299FE4F5587F012255
:034450007F0022C8
:0B45AF00302105C2217F01227F002285
:0100210022BC
:0645D400E4F558F5442255
:0A45BA00E4907570F0A3F0A3F02266
:104127002043616E457247495400200A0045727268
:104137004C656E43616E21000A002043616E457233
:1041470072434821000A205265714572722100C4EA
:1041570000C401C402C403C404C405C406C407C818
:1041670000C801C802C803C804C805C806C807C2F2
:1041770000C201C202C203C204C205C206C20700CE
:014187000037
:102F4900E59B541F6020200B1A7E417F271232AF68
:102F5900E59B541FFF7E007D031235657E417F315D
:102F69001232AFE4F59BE5BA30E010E4F5B375B180
:102F790080F5B2D223F555907C27F0E5CFF47003A4
:102F89000230A1752801E4F527E5CFF4552870032F
:102F990002308FE527C454F0F5B1E5B2547F6420BF
:102FA9006003023060E5B3540FF54A85BC46E5BDC0
:102FB900541FFF131313541FFFE5BD54E044184F6A
:102FC900F547E5BDC43354E0FFE5BE131313541FA1
:102FD9004FF548E5BEC43354E0FFE5BF131313545E
:102FE9001F4FF54985A34B85A34C85A34D85A34E5A
:102FF90085A34F85A35085A35185A352E4F5B2203B
:10300900190FE546547EB5460843BDF875B350809F
:103019000375B3D0E54A700AE546547EB546037F89
:103029000022301908E54630E7037F0022E54AD33C
:103039009408401D200B177E417F341232AFAF4AEE
:103049007E007D031235657E417F3F1232AF7F00DE
:1030590022E54A2405FF22E5B2549F6023200B2074
:103069007E417F411232AFAFB27E007D03123565DA
:10307900AFB37E007D031235657E417F3F1232AFCB
:10308900E4F5B275B3D0E52825E0F5280527E5274D
:0A309900C394085003022F927F0039
:0130A300220A
:1040C500907B0FE0C39464505675B180E4F5B3F569
:1040D500B28546BCE548C4135407FFE54754E04F95
:1040E500F5BDE54833333354F8FFE549C4135407A8
:1040F5004FF5BEE54933333354F8F5BF854BA385FA
:104105004CA3854DA3854EA3854FA38550A385510B
:10411500A38552A3E54A540F2450F5B375550AC239
:02412500232253
:1037230075B190E5B220E613200B107E417F4C1259
:1037330032AFAFB27E007D03123565E4F5B3F5B267
:10374300E50F30E615E4F50F907C42E02402F0E04B
:10375300904156937004907C42F07470250FF5826B
:10376300E43461F583E0702D907C42E0FFC31324C1
:1037730029F582E4347CF583E07005430F808015DE
:10378300E4F50F907C42E02402F0E0904156937000
:1037930004907C42F0E50F30E721907C42E0FF90FB
:1037A300415693F5BCE4F5BDEFA393FF3333335494
:1037B300F8F5BE75BF78430F4080367470250FF55A
:1037C30082E43461F583E0F5BC75BD807471250F27
:1037D300F582E43461F583E0FF33333354F8F5BE07
:1037E30075BF78050F050FE50FC394324003E4F569
:0537F3000F75B3502228
:0945C400EF6003C29622D2962298
:103E620043AB01C2E8C2EAE4FFEFC454F0F5B1C3C8
:103E7200EF64809488500575B3D08003E4F5B3E411
:103E8200F5B2F5BCF5BDF5BEF5BFF5C4F5C5F5C691
:103E9200F5C7F5A3F5A3F5A3F5A3F5A3F5A3F5A33C
:103EA200F5A30FBF0EC3907B0FE0FE25E0F5B475BE
:103EB200B50C75B66C75A11275AB0275C13E75C3B2
:103EC200FF75C203E4907C42F0750F80FF7F19906A
:103ED2007C29E4F0A3DFFCE4FF7F32906170E4F020
:033EE200A3DFFC5F
:013EE50022BA
:1014A0003E2A2C312CCFE0F0E0ECE5F2F0FB20F30B
:1014B000EFF0E0E2EBFFFEF9E5E3EE20EAEEEDF21D
:1014C000F0EEEBEBE5F0E020CACF20C8F1E5F2FC4E
:1014D0000A003E4C2C6B30312C25732C43EAEEF085
:1014E000EEF1F2FC20EDE020F8E8EDE52043414E7E
:1014F0002C30202D20353030EAE1283530EC292CF5
:1015000031202D203530EAE128353030EC290A0031
:1015100030202D20353030EAE1283530EC290031FB
:10152000202D203530EAE128353030EC29003E42CC
:101530002C6330312C2562752CC2F2EEF0E8F7ED09
:10154000FBE920EAEEEDF2F0EEEBEBE5F020EDE06A
:1015500020F8E8EDE50A003E2A2C312CCFE0F0E03F
:10156000ECE5F2F0FB20EFF0EEF2EEEAEEEBE0203D
:10157000C8F1E5F2FC20EFEE20EFEEF0F2F320529E
:10158000533233320A003E4C2C6B30352C256C75AF
:101590002CD1EAEEF0EEF1F2FC20EEE1ECE5EDE02C
:1015A00020EDE020EFEEF0F2F32C3130302C323031
:1015B000302C3330302C3630302C313230302C322D
:1015C0003430302C343830302C393630302C3139FE
:1015D0003230302C33383430302C35373630302CF4
:1015E0003131353230300A003E422C6B31302C25FF
:1015F00062752CCFF0EEF2EEEAEEEB20E1E5E720AB
:10160000ECE5F2EEEA20E2F0E5ECE5EDE80A003C7C
:1016100021003C6B30313D003C6330313D003C6B80
:1016200031303D003C6B30353D0043796354530A03
:1016300000537054530A0053705453210A005455F8
:101640000A00205455204D616B650A0043544949F6
:101650000A00435449540A0053705449540A005430
:10166000696D655449540A000A4173796E634F5598
:10167000543A00CEF820E4EBE8EDFB210A000A43DF
:101680005243204552523A20000A4173796E634911
:101690004E3A00C4EBE8EDE03F3F3F0A003F3F3FDA
:1016A0000A000089129B24AD36BF48C15AD36CE5AD
:1016B0007EF78108931AA52CB73EC940DB52ED6432
:1016C000FF76028B109926AF34BD4AC358D16EE71E
:1016D0007CF5830A9118A72EB53CCB42D950EF6612
:1016E000FD74048D169F20A932BB4CC55ED768E1FE
:1016F0007AF3850C971EA128B33ACD44DF56E960F2
:10170000FB72068F149D22AB30B94EC75CD56AE3DD
:1017100078F1870E951CA32AB138CF46DD54EB62D1
:10172000F97008811A932CA53EB740C952DB64EDCD
:1017300076FF89009B12AD24BF36C148D35AE56CB1
:10174000F77E0A8318912EA73CB542CB50D966EF9D
:1017500074FD8B029910AF26BD34C34AD158E76E91
:10176000F57C0C851E9728A13AB344CD56DF60E97D
:1017700072FB8D049F16A920BB32C54CD75EE16871
:10178000F37A0E871C952AA338B146CF54DD62EB5D
:1017900070F98F069D14AB22B930C74ED55CE36A51
:1017A000F17800112332465765748C9DAFBECADBB9
:1017B000E9F810013322564775649C8DBFAEDACB31
:1017C000F9E82130021367764455ADBC8E9FEBFAE1
:1017D000C8D93120120377665445BDAC9E8FFBEA11
:1017E000D8C94253617004152736CEDFEDFC8899C5
:1017F000ABBA5243716014053726DECFFDEC9889F1
:10180000BBAA6372405125340617EFFECCDDA9B8A0
:101810008A9B7362504135241607FFEEDCCDB9A8D0
:101820009A8B8495A7B6C2D3E1F008192B3A4E5F84
:101830006D7C9485B7A6D2C3F1E018093B2A5E4FB0
:101840007D6CA5B48697E3F2C0D129380A1B6F7E60
:101850004C5DB5A49687F3E2D0C139281A0B7F6E90
:101860005C4DC6D7E5F48091A3B24A5B69780C1D44
:101870002F3ED6C7F5E49081B3A25A4B79681C0D70
:101880003F2EE7F6C4D5A1B082936B7A48592D3C20
:101890000E1FF7E6D4C5B1A092837B6A58493D2C50
:0218A0001E0F19
:030023000237F8A9
:0D37F800C0E0C0F0C083C082C0D075D01802
:1038050030984AC298750B01AF99201A0BEF6402E4
:10381500703BD21AD2918035301C07C21C531F0F42
:10382500801CBF0904D21C8024BF031285616B6311
:103835006180536180C21A750B00C291800F741CA0
:103845002561F582E4346FF583EFF0056130996DFC
:10385500301B68E568B4FF0C7599020568756C0046
:10386500D2908057E568B560077599030568804B68
:10387500E568D39560400DC21BD21FC290E4FF12CC
:1038850045C48037E56C6009F5990568756C00805D
:103895002A741C2568F582E43470F583E0F56C64C0
:1038A50002600BE56C64036005E56CB40905759968
:0D38B500098008856C990568756C00C29942
:0B38C200D0D0D082D083D0F0D0E03214
:103B3A007BFF7A1479A0121904907B0FE070147538
:103B4A002EFF752F157530107BFF7A1479D2121952
:103B5A00048012752EFF752F1575301F7BFF7A149E
:103B6A0079D21219047BFF7A15792EA219E433F55A
:103B7A002E1219047BFF7A15795712190490746969
:103B8A00E0FEA3E0FFC3E49FFFE49EFEAB07FAE476
:103B9A00F9F8FF7E8C7D0AFC1222478F318E308D18
:103BAA002F8C2E7BFF7A1579861219047BFF7A15E2
:0C3BBA0079E8A21EE433F52E1219042253
:103397007E167F0F123CD4EF4E70037F0122E4901C
:1033A7007B0FF07E167F12123CD4EF4E601512454C
:1033B70076BF3106907B0F740AF0BF3206907B0F01
:1033C7007464F07E167F18123CD4EF4E600D1241E4
:1033D70088EC4D4E4F24FF92198002C2197E167F4A
:1033E7001E123CD4EF4E600D124188EC4D4E4F2417
:1033F700FF921E8002C21E7E167F24123CD4EF4E1F
:10340700600D1241888F298E288D278C26800BE42A
:10341700752980752825F527F526AB29AA28A92718
:10342700A8267F007E8C7D0A7C001222471222D9B3
:10343700907469EEF0A3EFF0E47F587E02FDFCABD9
:1034470029AA28A927A826D31222E75007756901B8
:10345700D21D8021E47F607E09FDFCAB29AA28A943
:1034670027A826D31222E75007756902C21D8005D7
:07347700756904C21D7F000E
:01347E00222B
:10364600E49061B3F09061A2F0906002F0C21BC2F8
:103656001FC21AC21CF568F560F508F561F50B90F6
:10366600746974FFF0A374F4F09061037402F0902F
:10367600616CF090616FF0C219E4907B0FF0C21D8F
:10368600123397E4F56A75F075E56AA42434F58279
:10369600E5F03468F583E4F0E56A75F00DA42404DA
:1036A600F582E43461F583E4F0F55F75F068E56A68
:1036B600A42429F582E5F03471F58375F00DE55FF4
:1036C600122335E4F0055FE55FB408DF056AE56AB5
:1036D600B408B3E4F56EF55AF55CF55DF567F56D7E
:1036E600F55FF55BF56AF566C2ADF5C9D2CDD2CC0C
:1036F600C2C9C2CAF5CDF5CC907469E0F5CBA3E09A
:10370600F5CA85CBCD85CACCD29ED29CD2CAC2ACD4
:0D371600C298C29975B81075B710D2AC22D8
:0100220022BB
:021F57008F27D2
:101F5900301D0EE546B44209E549640270030222C8
:101F69000AE54754E324DF70030220FE24DF7003EF
:101F79000220B11470030220B124E370030221335B
:101F89001470030221B51470030221E624E2602EC5
:101F99002460600302220A300C077E167F2A12325F
:101FA900AF301E03754A04E54875F00DA42404F505
:101FB90082E43461F5837D46AF2712298D22201EE4
:101FC90046E54875F00DA42404F582E43461F583EF
:101FD900E4F0300C077E167F311232AF75F00DE553
:101FE9005DA424DCF582E5F0346BF5837D46AF27EB
:101FF90012298D055D535D3FE55C655D6003022235
:102009000A055C535C3F22300C077E167F3712327B
:10201900AFE54875F00DA42409F582E43461F58330
:10202900E06404600302220AE54875F00DA4240463
:10203900F582E43461F583E546F07F01E54954070B
:10204900FEEFA806088002C333D8FCFFE549C39414
:1020590080502DE549541FFE131313541FFEE54804
:1020690075F00DA4240AF582E43461F583E5822E26
:10207900F582E43583F583E0FEEFF4FDEE5DF022B1
:10208900E549541FFE131313541FFEE54875F00D5F
:10209900A4240AF582E43461F583E5822EF582E40D
:1020A9003583F583E04FF022300C077E167F3E1210
:1020B90032AF90616EE06032E5466442702CE549CA
:1020C90064037026F0907AFB7402F0A37408F0A3FD
:1020D900E548F0A3F0A37401F0755606300B03022E
:1020E900220A7E167F421232AF2290711C7D46AFC2
:1020F9002712298D22300C077E167F4C1232AF75BC
:10210900F00DE55AA424B4F582E5F03461F5837D38
:1021190046AF2712298D055A535A7FE55A656E60D5
:102129000302220A056E536E7F22300C077E167F4A
:10213900521232AF201D4875F075E548A42441F5C7
:1021490082E5F03468F583E549541FFF1313543FC2
:1021590075F00D1223357D46AF2712298D75F0686C
:10216900E548A42429F582E5F03471F583E549545D
:102179001FFF1313543F75F00D122335E4F022436A
:10218900470143498075F068E548A42429F582E5AB
:10219900F03471F583E549543FFF1313543F75F04B
:1021A9000D1223357D467F0D12298D22300C077EB5
:1021B900167F581232AF75F068E548A42429F582D4
:1021C900E5F03471F583E549543FFF1313543F7526
:1021D900F00D1223357D467F0D12298D22201D21F8
:1021E900300C077E167F5F1232AF75F075E548A493
:1021F9002434F582E5F03468F5837D46AF2712294A
:012209008D47
:01220A0022B1
:103FDE008F2A90600363A20190701C63A201AF2A26
:103FEE0012299FE4F562F563852A6590701C63A221
:103FFE00019016A263A201AF65AE64AD63AC62120E
:10400E0029DB8F658E648D638C62741C252AF58284
:10401E00E43470F583E563F0741D252AF582E434EB
:10402E0070F583E562F0E52A2402F5607F01124502
:10403E00C47568FFD21BD299200B0D7E167F687C4B
:09404E00707D1CAB2A1230A42283
:10429B008E2B8F2C8F828E83E5822404F582E4355E
:1042AB0083F583E02405F568D3940E400B200B2A8D
:1042BB007E167F731232AF22852B83852C8263A2ED
:1042CB000174032566F582E43460F58363A201AFC4
:0B42DB006812299FE5682566F5662241
:1026D500756602E4F52AE52AC3956940030228C315
:1026E50090711CE0600D7E717F1C12429BE490711D
:1026F5001CF022E55D655C601B75F00DE55CA424AE
:10270500DCF582E5F0346BAF82FE12429B9061A24C
:102715007406F022E4F568E55E1470030227D4140C
:1027250070030227FC1470030228448000E4F55E60
:10273500301D030227CB75F075E56AA42434F582B4
:10274500E5F03468F583E06075E55B701875F07544
:10275500E56AA42434F582E5F03468AF82FE1242BE
:102765009B055B806175F075E56AA42437F582E504
:10277500F03468F583E0540FFFE55BD39F50237574
:10278500F075E56AA42434F582E5F03468F58375BF
:10279500F00DE55B122335AF82AE8312429B055BDC
:1027A5008024E4F55B75F075E56AA42434F582E5CB
:1027B500F03468F583E4F0056A536A078008E4F5A8
:1027C5005B056A536A07055EE56860030228BEE596
:1027D5005A656E601975F00DE56EA424B4F582E5B1
:1027E500F03461AF82FE12429B056E536E7F055E2B
:1027F500E56860030228BEE56775F00DA42404F5BD
:1028050082E43461F583E0602BE56775F00DA4245F
:1028150004F582E43461AF82FE12429BE56775F0F0
:102825000DA42404F582E43461F583E4F0056753CF
:10283500670780050567536707055EE568707A7564
:10284500F068E56DA42429F582E5F03471F583750A
:10285500F00DE55F122335E0604C75F068E56DA479
:102865002429F582E5F03471F58375F00DE55F12E5
:102875002335AF82AE8312429B75F068E56DA424C3
:1028850029F582E5F03471F58375F00DE55F1223C6
:1028950035E4F0055FE55FC39408401BE4F55F058B
:1028A5006D536D078011055FE55FC394084008E42B
:0E28B500F55F056D536D07055E052A0226DBF3
:0128C30022F2
:10248800E56775F00DA42404F582E43461F583E072
:1024980070050567536707201D1875F075E56AA470
:1024A8002434F582E5F03468F583E07005056A5355
:1024B8006A0775F068E56DA42429F582E5F03471A2
:1024C800F58375F00DE55F122335E07011055FE5C2
:1024D8005FC394084008E4F55F056D536D0730004D
:1024E8003690616EE0600214F0C20090616DE00405
:1024F800F09061B3E0600214F09061A2E0601814FB
:10250800F0E07013906002E004F0E0D39403400719
:10251800E4F0055C535C3FE508B40107E4F508D234
:102528001BD299E50BD394644007C21AE4F561F510
:102538000B301B0F90616DE0D39414400BC21BD27B
:102548001F8005E490616DF0201B2BE50870279033
:1025580061A2E070211226D5E566D394024017E403
:10256800906003F0A37419F0AF66123FDEE4F566DD
:10257800906000F0A3F0E56B70030226D4F527E421
:10258800F56BF562F563E527547FF565E52754801B
:10259800241CF582E4346FF58363A2019016A263CC
:1025A800A201AF65AE64AD63AC621229DB8F658EA4
:1025B800648D638C62E5275480241CF582E4346FB3
:1025C800AF82F5288F2953277FE5634562601D3068
:1025D8000B030226D47E167F7EAB27AD29AC2812CA
:1025E80030A47D03AF63AE6212356522200B0D7EE9
:1025F800167F89AB27AD29AC281230A4852982859E
:102608002883A3E024E760030226CAE52724FCF513
:1026180056C3940E40030226BCE556C394045003E7
:102628000226BC852982852883A3A3E0FF64447021
:1026380020E5292407F582E43528F583E0B4011163
:102648009061A2E06007E4F0055C535C3FE4F55656
:1026580022EFB44412E5292407F582E43528F583EE
:10266800E07004F55CF55D301D2F8529828528838F
:10267800A3A3E0B44223E5292406F582E43528F52E
:1026880083E0B40114E5292407F582E43528F583AD
:10269800E0700690616E7405F0E5292402FFE435C8
:1026A80028F5838F8263A201907AFB63A201AF565B
:1026B80012299F22E4F556200B127E167F931232C0
:0C26C800AF22200B077E167F9D1232AF60
:0126D40022E3
:103ABA00020911E493A3F8E493A34003F68001F208
:103ACA0008DFF48029E493A3F85407240CC8C3330D
:103ADA00C4540F4420C8834004F456800146F6DFDC
:103AEA00E4800B01020408102040809045CDE47E5A
:103AFA00019360BCA3FF543F30E509541FFEE493D1
:103B0A00A360010ECF54C025E060A840B8E493A397
:103B1A00FAE493A3F8E493A3C8C582C8CAC583CAC2
:103B2A00F0A3C8C582C8CAC583CADFE9DEE780BE7A
:0145D30000E7
:10220B0075F008758200EF2FFFEE33FECD33CDCC8A
:10221B0033CCC58233C5829BED9AEC99E58298400D
:10222B000CF582EE9BFEED9AFDEC99FC0FD5F0D6EA
:10223B00E4CEFBE4CDFAE4CCF9A88222B800C1B914
:10224B000059BA002DEC8BF084CFCECDFCE5F0CB52
:10225B00F97818EF2FFFEE33FEED33FDEC33FCEB8B
:10226B0033FB10D703994004EB99FB0FD8E5E4F946
:10227B00FA227818EF2FFFEE33FEED33FDEC33FC33
:10228B00C933C910D7059BE99A4007EC9BFCE99A27
:10229B00F90FD8E0E4C9FAE4CCFB2275F010EF2F6C
:1022AB00FFEE33FEED33FDCC33CCC833C810D7076C
:1022BB009BEC9AE899400AED9BFDEC9AFCE899F8A7
:0E22CB000FD5F0DAE4CDFBE4CCFAE4C8F9223A
:0E22D900C3E49FFFE49EFEE49DFDE49CFC2216
:1022E700EB9FF5F0EA9E42F0E99D42F0E89C45F04D
:0122F70022C4
:0C22F800ECF0A3EDF0A3EEF0A3EFF02259
:10230400A8828583F0D083D08212231B12231B1250
:10231400231B12231BE473E493A3C583C5F0C58375
:10232400C8C582C8F0A3C583C5F0C583C8C582C823
:012334002286
:0C233500A42582F582E5F03583F58322B3
:1018A200E53A242EF8E6053A22782B301702782EF4
:1018B200E475F0011223E80223412010EB7F2ED2BF
:1018C200108018EF540F2490D43440D4FF30140BFE
:1018D200EF24BFB41A0050032461FFE53B600215F8
:1018E2003B053EE53E7002053D30170D782BE47551
:1018F200F0011223E8EF0223870242E67403D217B3
:101902008003E4C217F53A8B2B8A2C892DE4F53B30
:10191200F53DF53EE53B60077F201218DD80F57549
:101922003CFFC211C210C212C213C215C216C218A3
:101932001218ABFF700D3017057F001218EEAF3E84
:10194200AE3D22B4255FC2D5C2141218ABFF24D01B
:10195200B40A00501A75F00A783B30D50508B6FF74
:101962000106C6A426F620D5047002D21380D9241B
:10197200CFB41A00EF5004C2E5D214021AEED2110B
:1019820080C6D21080C0D21280BCD2D580BAD21505
:1019920080B47F201218DD2012077401B53B00408D
:1019A200F11218A2FF1218DD021916D218D21680EF
:1019B200951218A2FB1218A2FA1218A2F94A4B7039
:1019C2000679BF7A1B7BFF20122EE53B602A7E0040
:1019D2008E8275830012235A60060EEE653C70F00B
:1019E200C2D5EBC0E0EAC0E0E9C0E0EE121B35D0A0
:1019F200E0F9D0E0FAD0E0FB122341FF60AAEBC08D
:101A0200E0EAC0E0E9C0E01218DDD0E02401F9D03C
:101A1200E03400FAD0E0FBE53C0460DCD53CD98040
:101A2200877BFF7A1B7931D212809C7910800279F0
:101A320008C216C2188008D2D5790A8004790AC26F
:101A4200D5E53C047002F53CE4FAFDFEFF1218A253
:101A5200FC7B082011131218A2FD7B1030100A1211
:101A620018A2FE1218A2FF7B20EC3382D592D55029
:101A720013C3E43010069FFFE49EFEE42011039D91
:101A8200FDE49CFCE4CBF8C211EC700CCFCECDCCC3
:101A9200E824F8F870F38017C3EF33FFEE33FEED5E
:101AA20033FDEC33FCEB33FB994002FB0FD8E9EB3F
:101AB200301105F8D0E0C448B211C0E00AEC4D4E36
:101AC2004F78207B0070C2EAB53C0040BCC0E012F7
:101AD2001B37D0F0D0E0201104C4C0E0C4B211C062
:101AE200F01218C6D0F0D5F0EB02191612244719DD
:101AF200B3531A2D5819844C1980421A314F1A398E
:0F1B0200441A39491999431A3F551A23461A2391
:101B1100451A23471BDF5019882D198C2E19AF2B1D
:101B210019902319AD201BC82A194848000019A78C
:101B31003F3F3F00790AA2D5201314301509B9108F
:101B4100020404B9080104A2D520160250010420A0
:101B510012689212B53B005034C0E07F2030131957
:101B61007F30A21272167215500F121B8EC212C252
:101B710016C215C2187F30800F301503E9C0E0127C
:101B810018DD301503D0E0F9D0E0B53BCC301517A6
:101B91007F30B9100C1218DD7F583014077F788020
:101BA10003B908031218DD3012057F2D0218DD7FFD
:101BB100202018F87F2B2016F322921280CF286E56
:101BC100756C6C2900D2111218A23011F8C211786B
:101BD1003B30D50108F60219482D504349581218D7
:101BE100A22403B405004001E4901BDA931218CE3D
:0D1BF100743A1218CED213753B04021A2D5F
:102AAD008B2A8A2B892CE4F536F535F534F533F57B
:102ABD0031F532E52E452F452D6012EBC0E0EAC011
:102ACD00E0E9C0E0AB2DAA2EA92F1223F8AB2A0501
:102ADD002CE52CAA2B7002052B14F9122341F53786
:102AED00C394094007E537D3940D40E1E5376420E1
:102AFD0060DBE537B42D054332038016E537B42B83
:102B0D0005433201800C74FF252CF52C74FF352BF9
:102B1D00F52BE53060046410703FAB2AAA2BA92C6D
:102B2D0012234164306009E530702E75300A80291A
:102B3D0090000112235AFF64786004EFB4581343D8
:102B4D0032017530107402252CF52CE4352BF52B44
:102B5D008007E5307003753008AB2A052CE52CAAEB
:102B6D002B7002052B14F9122341F537C3946140E4
:102B7D000AE537D3947A50035337DF74D02537F5F0
:102B8D0037C3940A400CE5379411406D74F925371D
:102B9D00F537E537D39530506043320185363B85A7
:102BAD00353A853439853338AF307E00E4FCFDABE2
:102BBD0036AA35A934A833122399C8ECC8C9EDC972
:102BCD00CAEECACBEFCBE4FCFDFEEB2537F536EEB6
:102BDD003AF535ED39F534EC38F533AF36AE35AD74
:102BED0034FCAB3BAA3AA939A838D31222E75003DB
:102BFD00022B66433204022B66E53220E003E480AB
:102C0D002DE52E452F452D601EAB2AE52C24FFF911
:102C1D00E52B34FFFAEBC0E0EAC0E0E9C0E0AB2DF4
:102C2D00AA2EA92F1223F8E53230E20774FFFFFE1A
:102C3D00FDFC22E532AF36AE35AD34AC3330E103B9
:042C4D000222D92264
:10234100BB010689828A83E0225002E722BBFE029A
:09235100E32289828A83E49322CD
:10235A00BB010CE58229F582E5833AF583E0225038
:10236A0006E92582F8E622BBFE06E92582F8E22282
:0D237A00E58229F582E5833AF583E493229C
:10238700BB010689828A83F0225002F722BBFE0135
:02239700F3222F
:10239900E88FF0A4CC8BF0A42CFCE98EF0A42CFCE3
:1023A9008AF0EDA42CFCEA8EF0A4CDA8F08BF0A461
:1023B9002DCC3825F0FDE98FF0A42CCD35F0FCEBC0
:1023C9008EF0A4FEA9F0EB8FF0A4CFC5F02ECD3985
:0F23D900FEE43CFCEAA42DCE35F0FDE43CFC22F2
:1023E800FAE6FB0808E6F925F0F618E6CA3AF622F6
:1023F800BB011A89828A83D0F0D0E0F8D0E0F9D006
:10240800E0FAD0E0FBE8C0E0C0F00224765016E91C
:10241800F8D083D082D0E0F9D0E0FAD0E0FBC082D7
:10242800C08302246DBBFE16E9F8D083D082D0E0C9
:0F243800F9D0E0FAD0E0FBC082C08302247F22FB
:10244700D083D082F8E4937012740193700DA3A324
:1024570093F8740193F5828883E473740293686038
:06246700EFA3A3A380DF38
:09246D00EBF608EAF608E9F62294
:09247600EBF0A3EAF0A3E9F02267
:09247F00EBF208EAF208E9F2228E
:00000001FF
